:020000040000FA
:0A0000000000000029EF00F040D0DE
:0800180093D09EA8FED7AD6E47
:100020001200096A086EFF0E0826092200D0D8A027
:100030001200030E076EE60E02D8F5D7076AFE0F10
:10004000066EE86A075AD8A012000000060600D023
:10005000F8D7006A4F0EAF6EB06A240EAC6E900EE9
:10006000AB6E00010F0EC16E070EB46E0FEE7EF088
:10007000ED6AE950EA10FCE1EF6AC69AC00E926E92
:10008000E00E936EC00E946E70D0F2A409D0F2947C
:100090000E4A0F2AD6CF0CF0D7CF0DF0817A11007F
:1000A0009EAA19D0060EAB1412E1E2CF29F0E1CFDF
:1000B00028F02A2A10EE36F02A50E126000EE2221D
:1000C000AECFE7FF29C0E2FF28C0E1FF1100AE502C
:1000D000AE50AB98AB8811002A502B5C14E02B2A51
:1000E000EACF07F0E9CF06F000EE36F02B50E92614
:1000F000000EEA22EF50276E07C0EAFF06C0E9FFB4
:10010000D880120004D0E868276ED8A01200120030
:100110002A6A2B6A9D8A9F8AF28EF28C12009D9A1F
:1001200000EE36F0010EF46EF36AF306000EF45A98
:10013000EE6AF450F310F9E12A6A2B6A9D8A1200E4
:10014000F29EE0CF38F6D8CF39F6E8CF3AF6F28E05
:100150000001A192B36AB26AF29E38C6E0FF39C6C6
:10016000D8FF3AC6E8FFF28E1000939A8A8A0A0EE8
:1001700058DF939A8A9A93948A9494968B96929045
:100180008990929289929294899492968996929863
:10019000899894908B9094928B9294948B9400EE87
:1001A0002EF0080EEE68E82EFDD71F6A05EE36F039
:1001B000010EF46EF36AF306000EF45AEE6AF45080
:1001C000F310F9E12C6A2D6AA3DFA9DFCD6AF2945E
:1001D000F28A870ED56EB16AA192A082B36AB26A22
:1001E000D08EA292B10EB16EF6D9E8EC06F008EC12
:1001F0000AF0B30E12DF420E10DF7F0E0EDFD6CFF5
:100200000CF0D7CF0DF068DF27C010F0B40E105CF3
:1002100006E3FE0E105C01E301D0126A0CD110AEB1
:1002200021D0126A830E105C05E110C012F0136831
:10023000146817D0930E105C05E110C012F0156819
:1002400016680FD0A30E105C05E110C012F01768FD
:10025000186807D0B30E105C04E110C012F01968E2
:100260001A68E8D0125202E1E6D0E4D0830E125CA4
:100270002DE1132803E110C013F026D010C014F0B4
:10028000180E135C1EE35B0E135C1BE20601366B5B
:10029000FF0E0C24026EFF0E0D20036E000E0E20CA
:1002A000046E000E0F20056E05C031F004C030F062
:1002B00003C02FF002C02EF013C037F68B8600016A
:1002C00001D0B9D01368B6D0B6D0B4D0930E125CBA
:1002D000D8A476D0152803E110C015F06FD010C057
:1002E00016F0165224E1180E155C1EE35B0E155C29
:1002F0001BE20601366BFF0E0C24026EFF0E0D2072
:10030000036E000E0E20046E000E0F20056E05C059
:1003100031F004C030F003C02FF002C02EF015C041
:1003200037F68B86000101D086D084D047D01FA03D
:1003300043D0180E155C3EE35B0E155C3BE215C026
:1003400036F6316830682F682E688B9604EE36F0EA
:10035000D8901534E926000EEA22EECF20F0EFCF38
:1003600021F020BE02D08B9401D08B8420BC02D01F
:100370008B9201D08B8220BA02D08B9001D08B80DF
:1003800020B802D0899801D0898820B602D08996F9
:1003900001D0898620B402D0899401D0898420B20A
:1003A00002D0899201D0898220B002D0899001D0F8
:1003B000898002D015683FD015683CD03CD03AD037
:1003C000A30E125C0AE1172803E110C017F003D056
:1003D00010C018F0A9D82FD02DD0B30E125C0AE1AE
:1003E000192803E110C019F003D010C01AF0A4D8E6
:1003F00022D020D0C30E125C07E11B2803E110C0FD
:100400001BF01B6818D016D0D30E125C07E11C2815
:1004100003E110C01CF08ED80ED00CD0E30E125C9D
:1004200009E11D2803E110C01DF003D010C01EF02B
:100430007FD801D03FD8020E265C34E222500C5CFB
:1004400023500D5824500E5825500F581EE3258E6A
:10045000265213E1899089928994899689988B9084
:100460008B928B94216A206A316830682F682E68DD
:100470000601376B8B96000107D0010E265C04E164
:10048000356834683368326815D80FAE0AD00F6A01
:100490000E6A0D6A0C6A00EE2EF0080EEE68E82E69
:1004A000FDD706D00FAE04D00F6A0E6A0D6A0C6A33
:1004B0008170A5D62668258E116A020E115C33E282
:1004C000D8901134E96EEA6AEA36E936EA362E0E39
:1004D000E926000EEA22EFCF02F0ECCF03F0ECCFDA
:1004E00004F0ECCF05F02250025C23500358245056
:1004F00004582550055815E2D8901134E96EEA6A7F
:10050000EA36E936EA362E0EE926000EEA22EFCF69
:1005100022F0ECCF23F0ECCF24F0ECCF25F011C08B
:1005200026F0112ACAE31200176812001B68120095
:100530001D6812001C6812000D0E195C18E18990EC
:1005400089928994899689988B908B928B94216A51
:10055000206A0601376B1A52000103E108EC0AF029
:1005600005D0010E1A5C02E1E5EC08F01BD0420E4A
:10057000195C08E11A5203E11F9016D802D08A8450
:100580001F8010D07B0E195C0CE1899089928994B0
:10059000899689988B908B928B94216A206A0601A8
:1005A000376B0001196812008A94899089928994A6
:1005B000899689988B908B928B94216A206A1F6A06
:1005C0000601376B00EE2EF0080EEE68E82EFDD720
:1005D0008B96000112000201376936695C0E396F93
:1005E0007A0E386F590E3B6F850E3A6F580E3D6F7D
:1005F000140E3C6F560E3F6FA90E3E6F550E416FA5
:10060000430E406F530E436FE30E426F520E456F21
:10061000890E446F510E476F350E466F4F0E496F6E
:10062000E60E486F4E0E4B6F9C0E4A6F4D0E4D6F8F
:10063000580E4C6F4C0E4F6F190E4E6F4A0E516F85
:10064000DF0E506F490E536FAA0E526F480E556F52
:100650007A0E546F470E576F4F0E566F460E596FF6
:10066000290E586F450E5B6F080E5A6F430E5D6F73
:10067000EB0E5C6F420E5F6FD30E5E6F410E616FCB
:10068000BF0E606F400E636FB00E626F3F0E656FFE
:10069000A50E646F3E0E676F9E0E666F3D0E696F0E
:1006A0009C0E686F3C0E6B6F9E0E6A6F3B0E6D6FFB
:1006B000A40E6C6F3A0E6F6FAE0E6E6F390E716FC7
:1006C000BC0E706F380E736FCE0E726F370E756F73
:1006D000E30E746F360E776FFD0E766F360E796F00
:1006E0001A0E786F350E7B6F3B0E7A6F340E7D6F6E
:1006F0005F0E7C6F330E7F6F870E7E6F320E816FC1
:10070000B20E806F310E836FE10E826F310E856FF6
:10071000140E846F300E876F490E866F2F0E896F0F
:10072000820E886F2E0E8B6FBE0E8A6F2D0E8D6F10
:10073000FD0E8C6F2D0E8F6F3F0E8E6F2C0E916FF6
:10074000850E906F2B0E936FCD0E926F2B0E956FC3
:10075000180E946F2A0E976F670E966F290E996F79
:10076000B80E986F290E9B6F0C0E9A6F280E9D6F16
:10077000620E9C6F270E9F6FBC0E9E6F270EA16F9F
:10078000180EA06F260EA36F760EA26F250EA56F12
:10079000D80EA46F250EA76F3C0EA66F240EA96F6E
:1007A000A20EA86F240EAB6F0B0EAA6F230EAD6FB7
:1007B000760EAC6F220EAF6FE40EAE6F220EB16FED
:1007C000540EB06F210EB36FC60EB26F210EB56F0F
:1007D0003B0EB46F200EB76FB20EB66F200EB96F1E
:1007E0002B0EB86F1F0EBB6FA60EBA6F1F0EBD6F1C
:1007F000240EBC6F1E0EBF6FA30EBE6F1E0EC16F08
:10080000250EC06F1D0EC36FA90EC26F1D0EC56FE2
:100810002E0EC46F1C0EC76FB60EC66F1C0EC96FAE
:100820003F0EC86F1B0ECB6FCB0ECA6F1B0ECD6F6A
:10083000580ECC6F1A0ECF6FE80ECE6F1A0ED16F16
:10084000790ED06F1A0ED36F0B0ED26F190ED56FB3
:10085000A00ED46F190ED76F360ED66F180ED96F43
:10086000CE0ED86F180EDB6F680EDA6F180EDD6FC4
:10087000030EDC6F170EDF6FA00EDE6F170EE16F39
:100880003F0EE06F160EE36FDF0EE26F160EE56FA0
:10089000800EE46F160EE76F240EE66F150EE96FFB
:1008A000C80EE86F150EEB6F6E0EEA6F150EED6F4A
:1008B000160EEC6F140EEF6FBF0EEE6F140EF16F8D
:1008C000690EF06F140EF36F150EF26F130EF56FC5
:1008D000C20EF46F130EF76F710EF66F130EF96FF1
:1008E000210EF86F120EFB6FD20EFA6F120EFD6F13
:1008F000840EFC6F120EFF6F380EFE6F110E030197
:10090000016FED0E006F110E036FA30E026F110E3B
:10091000056F5A0E046F110E076F120E066F100E40
:10092000096FCC0E086F100E0B6F870E0A6F100E3A
:100930000D6F420E0C6F0F0E0F6F0E69116FBD0E13
:10094000106F0F0E136F7C0E126F0F0E156F3D0E92
:10095000146F0E0E176FFE0E166F0E0E196FC00E6F
:10096000186F0E0E1B6F830E1A6F0E0E1D6F470E43
:100970001C6F0E0E1F6F0C0E1E6F0D0E216FD20E10
:10098000206F0D0E236F990E226F0D0E256F610ED5
:10099000246F0D0E276F2A0E266F0C0E296FF40E92
:1009A000286F0C0E2B6FBE0E2A6F0C0E2D6F8A0E49
:1009B0002C6F0C0E2F6F560E2E6F0C0E316F230EF8
:1009C000306F0B0E336FF10E326F0B0E356FC00EA2
:1009D000346F37693669A20E396FC30E386F9A0EBD
:1009E0003B6F460E3A6F960E3D6F320E3C6F920E85
:1009F0003F6F3A0E3E6F8E0E416F5D0E406F8A0E56
:100A0000436F9A0E426F860E456FF00E446F830E51
:100A1000476F5F0E466F7F0E496FE70E486F7C0E83
:100A20004B6F850E4A6F790E4D6F3B0E4C6F760EF5
:100A30004F6F070E4E6F720E516FE80E506F6F0EB4
:100A4000536FDF0E526F6C0E556FEA0E546F6A0EC5
:100A5000576F0A0E566F670E596F3C0E586F640E33
:100A60005B6F820E5A6F610E5D6FDA0E5C6F5F0E08
:100A70005F6F440E5E6F5C0E616FBF0E606F5A0E4B
:100A8000636F4C0E626F570E656FE90E646F550E03
:100A9000676F960E666F530E696F686F510E6B6FBE
:100AA000200E6A6F4E0E6D6FFB0E6C6F4C0E6F6FEB
:100AB000E50E6E6F4A0E716FDC0E706F480E736F2D
:100AC000E20E726F460E756FF50E746F450E776FFE
:100AD000150E766F430E796F420E786F410E7B6F65
:100AE0007B0E7A6F3F0E7D6FC00E7C6F3E0E7F6F68
:100AF000100E7E6F3C0E816F6D0E806F3A0E836F0D
:100B0000D40E826F390E856F460E846F370E876F55
:100B1000C20E866F360E896F490E886F340E8B6F4A
:100B2000DA0E8A6F330E8D6F740E8C6F320E8F6FEC
:100B3000180E8E6F300E916FC50E906F2F0E936F43
:100B40007B0E926F2E0E956F3A0E946F2D0E976F4F
:100B5000020E966F2B0E996FD10E986F2A0E9B6F17
:100B6000A90E9A6F290E9D6F880E9C6F280E9F6F9D
:100B70006F0E9E6F270EA16F5E0EA06F260EA36FE5
:100B8000530EA26F250EA56F500EA46F240EA76FF3
:100B9000540EA66F230EA96F5E0EA86F220EAB6FC8
:100BA0006F0EAA6F210EAD6F860EAC6F200EAF6F69
:100BB000A30EAE6F1F0EB16FC60EB06F1E0EB36FD9
:100BC000EF0EB26F1E0EB56FB46F1D0EB76F520EE3
:100BD000B66F1C0EB96F8C0EB86F1B0EBB6FCB0EB1
:100BE000BA6F1B0EBD6F0F0EBC6F1A0EBF6F580E83
:100BF000BE6F190EC16FA50EC06F180EC36FF80E31
:100C0000C26F180EC56F4F0EC46F170EC76FAB0EB5
:100C1000C66F170EC96F0A0EC86F160ECB6F6F0E18
:100C2000CA6F150ECD6FD70ECC6F150ECF6F430E5A
:100C3000CE6F140ED16FB30ED06F140ED36F270E7C
:100C4000D26F130ED56F9F0ED46F130ED76F1A0E7F
:100C5000D66F120ED96F990ED86F120EDB6F1B0E66
:100C6000DA6F110EDD6FA10EDC6F110EDF6F290E32
:100C7000DE6F100EE16FB50EE06F100EE36F440EE5
:100C8000E26F0F0EE56FD60EE46F0F0EE76F6B0E7F
:100C9000E66F0F0EE96F030EE86F0E0EEB6F9D0E01
:100CA000EA6F0E0EED6F3A0EEC6F0D0EEF6FDA0E6F
:100CB000EE6F0D0EF16F7C0EF06F0D0EF36F210EC7
:100CC000F26F0C0EF56FC80EF46F0C0EF76F720E0C
:100CD000F66F0C0EF96F1E0EF86F0B0EFB6FCC0E3D
:100CE000FA6F0B0EFD6F7C0EFC6F0B0EFF6F2E0E5E
:100CF000FE6F0A0E0401016FE30E006F0A0E036F10
:100D0000990E026F0A0E056F510E046F0A0E076FDF
:100D10000B0E066F090E096FC80E086F090E0B6FD8
:100D2000850E0A6F090E0D6F450E0C6F090E0F6FC1
:100D3000060E0E6F080E116FC90E106F080E136F9E
:100D40008E0E126F080E156F540E146F080E176F6B
:100D50001C0E166F070E196FE50E186F070E1B6F2E
:100D6000AF0E1A6F070E1D6F7B0E1C6F070E1F6FE5
:100D7000490E1E6F070E216F170E206F060E236F90
:100D8000E70E226F060E256FB90E246F060E276F31
:100D90008B0E266F060E296F5F0E286F060E2B6FC7
:100DA000340E2A6F060E2D6F0A0E2C6F050E2F6F54
:100DB000E10E2E6F050E316FB90E306F050E336FD9
:100DC000930E326F050E356F6D0E346F00011200F9
:100DD000040E0101396F880E386F040E3B6FA60EAA
:100DE0003A6F040E3D6FB60E3C6F040E3F6FC60E99
:100DF0003E6F040E416FD60E406F040E436FE60E39
:100E0000426F040E456FF60E446F050E476F070ED6
:100E1000466F050E496F170E486F050E4B6F280E73
:100E20004A6F050E4D6F390E4C6F050E4F6F4B0E0E
:100E30004E6F050E516F5D0E506F050E536F6E0EA7
:100E4000526F050E556F800E546F050E576F930E3F
:100E5000566F050E596FA50E586F050E5B6FB80ED5
:100E60005A6F050E5D6FCB0E5C6F050E5F6FDF0E68
:100E70005E6F050E616FF20E606F060E636F626F3C
:100E8000656F1A0E646F060E676F2E0E666F060E84
:100E9000696F430E686F060E6B6F580E6A6F060E11
:100EA0006D6F6D0E6C6F060E6F6F830E6E6F060E9C
:100EB000716F980E706F060E736FAE0E726F060E26
:100EC000756FC40E746F060E776FDB0E766F060EAD
:100ED000796FF20E786F070E7B6F090E7A6F070E2F
:100EE0007D6F210E7C6F070E7F6F380E7E6F070EB1
:100EF000816F500E806F070E836F690E826F070E31
:100F0000856F810E846F070E876F9A0E866F070EAE
:100F1000896FB40E886F070E8B6FCD0E8A6F070E28
:100F20008D6FE70E8C6F080E8F6F020E8E6F080E9E
:100F3000916F1D0E906F080E936F380E926F080E12
:100F4000956F530E946F080E976F6F0E966F080E85
:100F5000996F8B0E986F080E9B6FA70E9A6F080EF5
:100F60009D6FC40E9C6F080E9F6FE10E9E6F080E62
:100F7000A16FA069090EA36F1D0EA26F090EA56FC8
:100F80003B0EA46F090EA76F5A0EA66F090EA96F2C
:100F9000790EA86F090EAB6F990EAA6F090EAD6F8F
:100FA000B90EAC6F090EAF6FD90EAE6F090EB16FEF
:100FB000FA0EB06F0A0EB36F1B0EB26F0A0EB56F4A
:100FC0003D0EB46F0A0EB76F5F0EB66F0A0EB96FA3
:100FD000820EB86F0A0EBB6FA50EBA6F0A0EBD6FF8
:100FE000C80EBC6F0A0EBF6FEC0EBE6F0B0EC16F4A
:100FF000110EC06F0B0EC36F360EC26F0B0EC56F96
:101000005B0EC46F0B0EC76F810EC66F0B0EC96FE0
:10101000A70EC86F0B0ECB6FCE0ECA6F0B0ECD6F27
:10102000F50ECC6F0C0ECF6F1D0ECE6F0C0ED16F68
:10103000460ED06F0C0ED36F6F0ED26F0C0ED56FA5
:10104000980ED46F0C0ED76FC20ED66F0C0ED96FE0
:10105000ED0ED86F0D0EDB6F180EDA6F0D0EDD6F13
:10106000430EDC6F0D0EDF6F700EDE6F0D0EE16F45
:101070009C0EE06F0D0EE36FCA0EE26F0D0EE56F72
:10108000F80EE46F0E0EE76F260EE66F0E0EE96F98
:10109000550EE86F0E0EEB6F850EEA6F0E0EED6FBC
:1010A000B60EEC6F0E0EEF6FE70EEE6F0F0EF16FD8
:1010B000180EF06F0F0EF36F4B0EF26F0F0EF56FF1
:1010C0007E0EF46F0F0EF76FB10EF66F0F0EF96F05
:1010D000E60EF86F100EFB6F1B0EFA6F100EFD6F11
:1010E000500EFC6F100EFF6F870EFE6F100E020188
:1010F000016FBE0E006F100E036FF60E026F110E21
:10110000056F2E0E046F110E076F680E066F110E1D
:10111000096FA20E086F110E0B6FDC0E0A6F120E14
:101120000D6F180E0C6F120E0F6F540E0E6F120E05
:10113000116F910E106F120E136FCF0E126F130EF0
:10114000156F0E0E146F130E176F4D0E166F130ED4
:10115000196F8E0E186F130E1B6FCF0E1A6F140EB1
:101160001D6F110E1C6F140E1F6F540E1E6F140E88
:10117000216F980E206F140E236FDC0E226F150E58
:10118000256F220E246F150E276F680E266F150E21
:10119000296FB00E286F150E2B6FF80E2A6F160EE2
:1011A0002D6F410E2C6F160E2F6F8C0E2E6F160E9C
:1011B000316FD70E306F170E336F230E326F170E4D
:1011C000356F700E346F00011200116A160E115C3B
:1011D0000BE204EE36F0D8901134E926000EEA2234
:1011E000EE6AEF6A112AF2E30401636B626B800E10
:1011F000656F646BC00E676F666BE00E696F686B3E
:10120000F00E6B6F6A6BF80E6D6F6C6BFC0E6F6F90
:101210006E6BFE0E716F706B7369726B7569800E09
:10122000746F7769C00E766F7969E00E786F7B6BAB
:101230007A6B800E7D6F7C6BC00E7F6F7E6BE00ED5
:10124000816F806BF00E836F826BF80E856F846BFD
:10125000FC0E876F866BFE0E896F886B8B698A6BBD
:101260008D69800E8C6F8F69C00E8E6F9169E00E54
:10127000906F936B926B800E956F946BC00E976F0F
:10128000966BE00E996F986BF00E9B6F9A6BF80E51
:101290009D6F9C6BFC0E9F6F9E6BFE0EA16FA06BF3
:1012A000A369A26BA569800EA46FA769C00EA66F83
:1012B000A969E00EA86FAB69F00EAA6FAD69F80ED0
:1012C000AC6F96C402F097C403F003C0AFF402C041
:1012D000AEF498C402F099C403F003C0B1F402C0A4
:1012E000B0F49AC402F09BC403F003C0B3F402C08C
:1012F000B2F49CC402F09DC403F003C0B5F402C074
:10130000B4F49EC402F09FC403F003C0B7F402C05B
:10131000B6F4A0C402F0A1C403F003C0B9F402C043
:10132000B8F4A2C402F0A3C403F003C0BBF402C02B
:10133000BAF4A4C402F0A5C403F003C0BDF402C013
:10134000BCF4A6C402F0A7C403F003C0BFF402C0FB
:10135000BEF4A8C402F0A9C403F003C0C1F402C0E3
:10136000C0F4AAC402F0ABC403F003C0C3F402C0CB
:10137000C2F4ACC402F0ADC403F003C0C5F402C0B3
:10138000C4F4C769FC0EC66FC969FE0EC86FCB698D
:10139000CA69F80ECD6FCC6BFC0ECF6FCE6BFE0E14
:1013A000D16FD06BD369D26BD569800ED46FD769FA
:1013B000C00ED66FD969E00ED86FDB69F00EDA6F18
:1013C000DD69F80EDC6FDF69FC0EDE6FE169FE0E91
:1013D000E06FE369E269F80EE56FE46BFC0EE76F1E
:1013E000E66BFE0EE96FE86BEB69EA6B5B0E116E64
:1013F0000001800E115C0BE204EE36F0D89011343F
:10140000E926000EEA22EE6AEF6A112AF1E31200E1
:10141000116A160E115C0BE204EE36F0D89011340E
:10142000E926000EEA22EE6AEF6A112AF2E30401CD
:10143000636B626B800E656F646B400E676F666BEB
:10144000200E696F686B100E6B6F6A6B080E6D6F04
:101450006C6B040E6F6F6E6B020E716F706B010E12
:10146000736F726B756B800E746F776B400E766F57
:10147000796B200E786F7B6B7A6B800E7D6F7C6B47
:10148000400E7F6F7E6B200E816F806B100E836F1E
:10149000826B080E856F846B040E876F866B020E5D
:1014A000896F886B010E8B6F8A6B8D6B800E8C6FD2
:1014B0008F6B400E8E6F916B200E906F936B926BC3
:1014C000800E956F946B400E976F966B200E996F00
:1014D000986B100E9B6F9A6B080E9D6F9C6B040EA1
:1014E0009F6F9E6B020EA16FA06B010EA36FA26B8C
:1014F000A56B800EA46FA76B400EA66FA96B200E84
:10150000A86FAB6B100EAA6FAD6B080EAC6F96C4D4
:1015100002F097C403F003C0AFF402C0AEF498C465
:1015200002F099C403F003C0B1F402C0B0F49AC44D
:1015300002F09BC403F003C0B3F402C0B2F49CC435
:1015400002F09DC403F003C0B5F402C0B4F49EC41D
:1015500002F09FC403F003C0B7F402C0B6F4A0C405
:1015600002F0A1C403F003C0B9F402C0B8F4A2C4ED
:1015700002F0A3C403F003C0BBF402C0BAF4A4C4D5
:1015800002F0A5C403F003C0BDF402C0BCF4A6C4BD
:1015900002F0A7C403F003C0BFF402C0BEF4A8C4A5
:1015A00002F0A9C403F003C0C1F402C0C0F4AAC48D
:1015B00002F0ABC403F003C0C3F402C0C2F4ACC475
:1015C00002F0ADC403F003C0C5F402C0C4F4C76B9D
:1015D000040EC66FC96B020EC86FCB6B010ECA6FCB
:1015E000080ECD6FCC6B040ECF6FCE6B020ED16F99
:1015F000D06B010ED36FD26BD56B800ED46FD76BCF
:10160000400ED66FD96B200ED86FDB6B100EDA6FE1
:10161000DD6B080EDC6FDF6B040EDE6FE16B020E1C
:10162000E06FE36B010EE26F080EE56FE46B040EF2
:10163000E76FE66B020EE96FE86B010EEB6FEA6B8A
:101640005B0E116E0001800E115C0BE204EE36F0B1
:10165000D8901134E926000EEA22EE6AEF6A112AC8
:06166000F1E31200FFD7C8
:020000040030CA
:0300010006160ED2
:020005008580F4
:060008000FC00FE00F40E5
:00000001FF
